:020000040000FA
:1000000000308B0000308500003086008316C5303C
:10001000810010308500F030860083120030980097
:1000200099000D3084008001840A041E1328841E68
:100030001328851505119801990196019701A601CC
:10004000A701A801AA3090009611172217221722A3
:100050003330062233300622323006222C3006227C
:10006000063006220C30062201300622023006221B
:10007000172217220130F222920006148511061E63
:10008000432801309206861E472892141211061F3B
:100090004B2812159210861F4F28121192108515A9
:1000A0000610DE229218762812197E2805224C307E
:1000B00007224F30072243300722203007225330D7
:1000C00007225030072220300722443007222030F8
:1000D00007223130072232300722333007223430F2
:1000E000072220300722463007229028052254306C
:1000F00007224F300722473007225D2805224C3067
:1001000007224F3007224B3007222030072246308B
:100110000722533007222030072252300722672857
:10012000E22014212D215721A721FF21A220CD203B
:10013000A220CD20CD209F0D9F1E90289F0103104F
:100140001F1490282E089A000830940005109A0D6C
:10015000DC20031C0514D3200514DC20940BA628F6
:100160000510DC20971E0514D3200514DC20051093
:10017000DC20171F0514D3200514DC2011089A0079
:100180000830940005109A0DDC20031C0514D320C0
:100190000514DC20940BC2280800263093002D2182
:1001A000930BCF28080005309300000000000000EA
:1001B0002D21930BD8280800043093000000930BE6
:1001C000DE280800CA22121C032212180522303031
:1001D00007221808303E07221908303E0722203037
:1001E0000722150807222D080722203007223C305D
:1001F0001718023E072220300722203097180A3EA7
:100200000722203017190A3E0722203097190A3E8C
:1002100007222030171A0A3E0722203007222030FA
:10022000971A0A3E0722080085119B0104309C00A2
:1002300086010314860D0310061A2A299B0A861AC2
:100240002A299B0A061B2A299B0A861B2A299B0A04
:100250009C0B1A298515860108002810A810851501
:100260000608C039A6000319A81427020319281488
:10027000C03026020319A814A81C472928185029A1
:10028000281D9E0A28199E032608A7000800281189
:100290002708A606A61B281500000000000008007D
:1002A00000000000000000000000000008001B1A11
:1002B000A3291B08083EF2229B000A301B020318E8
:1002C00075291619080016186D29161496141B089E
:1002D0009800703099003E22080096180800161009
:1002E0001B0899001615202208009619A4299615B6
:1002F0000B301B02031D80299E0101309706A429A3
:100300000A301B02031D872920309706A4290C30D0
:100310001B02031D8E2902309706A4290D301B02F3
:10032000031D952904309706A4290E301B02031DD6
:100330009C2908309706A4290F301B02031DA4290D
:1003400010309706A4299611961016110800961DD4
:10035000B0290B301B02031DB029C03091000800EA
:10036000A00103101F1CB829171CB8291030A000C9
:100370009F1CBE29203097186030A0001F1DC42983
:10038000303017197030A0009F1DCA2940309719CE
:100390008030A0001F1ED0295030171A9030A000C6
:1003A000C0301E0203189E011C301E02031CDA29F5
:1003B0001C309E0003111E03031DE12904309E0022
:1003C000E529FD301E0703199E011E08A900291802
:1003D000F029A90CA913971A1717971E1713F629B6
:1003E000A90CA913971A1713971E17172908A00706
:1003F00003308A00200800238A0191000800051EAE
:1004000008002D21FF29C030062A80308511A40064
:100410001430A300A30B0A2A10221022851508000D
:10042000A40E24080F3986000515051108000A30AE
:10043000A5008B010B1D1A2A0B11A50B1A2A080007
:10044000AF011808A1000310210DA10EA10C210776
:10045000190790009D0032301D02031C332A023020
:10046000AF0032309D0203109D0D9D0DB5221F304F
:100470001E02031C08009E0197010800AF0110082E
:100480009D0032301D02031C492A0230AF00323079
:100490009D0203109D0D9D0DA92208008316851451
:1004A0008312080085108316851083120800061435
:1004B000080006100800572200000000000000009D
:1004C00059220000000000000000080059224E22BE
:1004D00057225222592200000000000000000800AC
:1004E0005922522257224E225922000000000000B9
:1004F000000008004E225B22080052225B22080006
:10050000AB000830AA000310AB0D03188B2A52224F
:100510005B224E228D2A4E225B22AA0B832A7A224C
:1005200008000830AA004E225722000000000000F8
:1005300000000000851C9E2A03149F2A0310AC0DA6
:1005400059220000000000000000AA0B942A2C0889
:1005500008006622A0302F0780221D0880221E0876
:10056000802217088022702208006622A0302F0700
:1005700080221D0880226622A1302F07802291222E
:100580009E007D22912297007D229122AE007A2248
:100590007022080003111E08031DFD3EA200A101E8
:1005A0000A302202031CD72AA200A10AD02A21085D
:1005B000303E95002208303EAD0008001208880049
:1005C0000130890083168B130812881108155530E5
:1005D0008900AA308900881408118818ED2A83122E
:1005E0008B17080089008316081483120808080076
:100600008207113491343134B13419349934393486
:10061000B934123492343234B2341A349A343A340B
:10062000BA344534C5346534E5344D34CD346D3495
:10063000ED344634C6346634E6344E34CE346E344B
:10064000EE345034D0347034E4345834D834783400
:10065000F8345234D2347234F2345A34DA347A34CC
:10066000FA34043484342434A4344C348C342C349C
:10067000AC34063486342634A6340E348E342E340C
:10068000AE34143494343434B4341C349C346C3468
:10069000BC34163496343634B6341E349E343E346C
:1006A000BE345434D4347434F4345C34DC347C34A8
:1006B000EC345634D6347634F6345E34DE347E345C
:1006C000FE345134D1347134F1345934D93479345D
:1006D000F9345334D3347334B3345B34DB347B3484
:1006E000FB34053485342534A5340D348D342D3454
:1006F000AD34073487342734A7341B348F342F3478
:10070000AF34153495343534B5341D349D343D340F
:10071000BD34173497343734B7341F349F343B34E7
:10072000BF345534D5347534F5345D34DD347D341F
:10073000FD345734D7347734F7345F34DF347F34C3
:02074000BB34C8
:02400E00F93F78
:1042000000000000000000000000000000000000AE
:104210000100020003000F000400050006000E006C
:104220000700080009000D000A0000000B000C0048
:10423000000000000000000000000000000000007E
:10424000000000000000000000000000000000006E
:10425000000000000000000000000000000000005E
:10426000000000000000000000000000000000004E
:10427000000000000000000000000000000000003E
:00000001FF
